:0200000480007A
:100000006F00C004732F2034930F8000630AFF0336
:10001000930F90006306FF03930FB0006302FF038A
:10002000170F0080130F0FFE63040F0067000F000F
:10003000732F203463540F006F004000136E9E53E3
:10004000171F00002320CFFD6FF09FFF732540F1A5
:100050006310050073251030635805000F00F00F82
:10006000130E100073000000130E00009702000032
:10007000938282F973905230735020307350303035
:1000800073504030970200809382C2F7638C020065
:10009000739052109302B01A739022307323203061
:1000A000E39E62F873500030970200009382420191
:1000B00073901234732540F173002030B70001FFB4
:1000C000938000F037110F0F1301F1F0B3C120003E
:1000D000B7FE0FF0938EFE00130E20006390D14BFD
:1000E000B710F00F938000FF37F1F0F01301010F0C
:1000F000B3C12000B70E01FF938E0EF0130E300037
:10010000639ED147B700FF009380F00F37110F0FA8
:100110001301F1F0B3C12000B71EF00F938E0EFF54
:10012000130E4000639CD145B7F00FF09380F000B0
:1001300037F1F0F01301010FB3C12000B70EFF003B
:10014000938EFE0F130E5000639AD143B70001FF48
:10015000938000F037110F0F1301F1F0B3C02000AE
:10016000B7FE0FF0938EFE00130E60006398D0412F
:10017000B70001FF938000F037110F0F1301F1F06A
:1001800033C12000B7FE0FF0938EFE00130E7000F7
:100190006316D13FB70001FF938000F0B3C0100099
:1001A000930E0000130E8000639AD03D13020000EE
:1001B000B70001FF938000F037110F0F1301F1F02A
:1001C000B3C1200013830100130212009302200028
:1001D000E31052FEB7FE0FF0938EFE00130E900058
:1001E000631ED33913020000B710F00F938000FF95
:1001F00037F1F0F01301010FB3C12000130000002C
:10020000138301001302120093022000E31E52FC2C
:10021000B70E01FF938E0EF0130EA0006310D337BC
:1002200013020000B700FF009380F00F37110F0F8B
:100230001301F1F0B3C1200013000000130000000F
:10024000138301001302120093022000E31C52FCEE
:10025000B71EF00F938E0EFF130EB0006310D33352
:1002600013020000B70001FF938000F037110F0F59
:100270001301F1F0B3C12000130212009302200019
:10028000E31252FEB7FE0FF0938EFE00130EC00075
:100290006396D12F13020000B710F00F938000FF78
:1002A00037F1F0F01301010F13000000B3C120007B
:1002B0001302120093022000E31052FEB70E01FF5A
:1002C000938E0EF0130ED000639AD12B1302000010
:1002D000B700FF009380F00F37110F0F1301F1F0FB
:1002E0001300000013000000B3C12000130212002D
:1002F00093022000E31E52FCB71EF00F938E0EFFF8
:10030000130EE000639CD12713020000B70001FF29
:10031000938000F01300000037110F0F1301F1F06C
:10032000B3C120001302120093022000E31052FE1A
:10033000B7FE0FF0938EFE00130EF0006390D125F0
:1003400013020000B710F00F938000FF13000000AD
:1003500037F1F0F01301010F13000000B3C12000CA
:100360001302120093022000E31E52FCB70E01FF9D
:10037000938E0EF0130E00016392D1211302000040
:10038000B700FF009380F00F13000000130000007F
:1003900037110F0F1301F1F0B3C120001302120047
:1003A00093022000E31E52FCB71EF00F938E0EFF47
:1003B000130E10016394D11D1302000037110F0FAB
:1003C0001301F1F0B70001FF938000F0B3C12000EA
:1003D0001302120093022000E31252FEB7FE0FF048
:1003E000938EFE00130E2001639AD11913020000B0
:1003F00037F1F0F01301010FB710F00F938000FFF9
:1004000013000000B3C12000130212009302200069
:10041000E31052FEB70E01FF938E0EF0130E300163
:10042000639ED1151302000037110F0F1301F1F075
:10043000B700FF009380F00F1300000013000000CE
:10044000B3C120001302120093022000E31E52FCED
:10045000B71EF00F938E0EFF130E40016390D11361
:100460001302000037110F0F1301F1F01300000009
:10047000B70001FF938000F0B3C120001302120007
:1004800093022000E31052FEB7FE0FF0938EFE00A1
:10049000130E50016394D10F1302000037F1F0F0F6
:1004A0001301010F13000000B710F00F938000FF3D
:1004B00013000000B3C120001302120093022000B9
:1004C000E31E52FCB70E01FF938E0EF0130E600177
:1004D0006396D10B1302000037110F0F1301F1F0D7
:1004E0001300000013000000B700FF009380F00F1E
:1004F000B3C120001302120093022000E31E52FC3D
:10050000B71EF00F938E0EFF130E70016398D10784
:10051000B70001FF938000F033411000B70E01FFD8
:10052000938E0EF0130E8001631AD105B700FF0001
:100530009380F00F33C10000B70EFF00938EFE0FC3
:10054000130E9001631CD103B3400000930E000012
:10055000130EA0016394D003B710111193801011F2
:10056000372122221301212233C02000930E0000E4
:10057000130EB0016314D001631CC0010F00F00F13
:1005800063000E00131E1E00136E1E007300000099
:100590000F00F00F130E100073000000731000C066
:1005A000000000000000000000000000000000004B
:1005B000000000000000000000000000000000003B
:0405C0000000000037
:1010000000000000000000000000000000000000E0
:1010100000000000000000000000000000000000D0
:1010200000000000000000000000000000000000C0
:1010300000000000000000000000000000000000B0
:081040000000000000000000A8
:040000058000200057
:00000001FF
